:020000020000FC
:020000009DC0A1
:10000C0000C00FB617EE12BF739586FF0BC0089495
:10001C00809B88944795783019F4112719BF806814
:10002C000FBE1895713011F49198FACF7A3029F4EB
:10003C00919A112719BF8064F3CF40FD919A40FF2C
:10004C0091984695EDCF80E412E013BF899A889879
:10005C0008958827772712E019BF86FFFECF0895F1
:10006C00809BFECF8099FECF13EE12BF12E018BF1B
:10007C0019BF772787FFFECF8F7708952FEF2A952B
:10008C00F1F71A95D9F70895332718E0F0E0331FEC
:10009C0010F4C69A01C0C698FF0FB599F160C79AC3
:1000AC0026E02A95F1F7C79823E02A95F1F71A95DF
:1000BC0071F73F2F089500001FED17BBC798C49A26
:1000CC001FEFDCDFC4981FEFD9DF3CEADEDF33E53E
:1000DC00DCDF0032B8F00023AAF0A0E2D5DF333524
:1000EC0099F030E0D2DFC79A26E02A95F1F7C7984D
:1000FC0023E02A95F1F73CEAC8DF33E5C6DFAA9581
:10010C0069F702C030E0C1DF30E0BFDF10E1B6DFDD
:10011C00089541E49EDF46E59CDF42E59ADF40E22C
:10012C0098DF49E496DF43E594DF40E592DF0895DC
:10013C000FED0DBF11271BBF1FEF12BBC49A18BBCD
:10014C0010E117BB80DF78948BDF4B31E9F344353A
:10015C0019F486DF042F41C1433511F4DADFF4CFF3
:10016C00463529F442E375DF42E373DFEDCF4637C2
:10017C0029F441E66EDF40E66CDFE6CF443729F523
:10018C0045E567DF46E565DF43E163DF40E261DFBC
:10019C0048E25FDF48E35DDF48E45BDF4CE459DFB6
:1001AC0044E357DF40E355DF4CE653DF48E651DFCD
:1001BC0045E64FDF40E64DDF44E64BDF41E449DFE7
:1001CC0042E447DF40E045DFBFCF403719F443E559
:1001DC0040DFBACF413619F449E53BDFB5CF48379C
:1001EC0009F4FBC0493709F4F8C0053509F10635A7
:1001FC00F9F00331E9F00032D9F00832C9F00833D4
:10020C00B9F00834A9F00C3499F0043389F00033B8
:10021C0079F00C3669F0083659F0053649F000369D
:10022C0039F0043629F0023419F0013409F0D2C047
:10023C00403511F440DFD1C0433471F411DF38E4A0
:10024C0024DF362F22DF352F20DF342F1EDF11E085
:10025C002227510F621F0BC04336B1F401DF30E48B
:10026C0014DF362F12DF352F10DF342F0EDF013461
:10027C0051F0053641F0023431F0003621F00436ED
:10028C0011F010E2FBDEA9C0423599F438E2FDDE34
:10029C00362FFBDE352FF9DEF7DE432FDADE30E2C8
:1002AC00F4DE362FF2DE352FF0DEEEDE432FD1DE1C
:1002BC0024C0413429F4D4DE642FD2DE542F8DC0F7
:1002CC00443481F4CDDE30ECE0DE362FDEDE352F2B
:1002DC00DCDE342FDADE10E2D1DE11E02227510F02
:1002EC00621F7BC0443671F430EACFDE362FCDDE90
:1002FC00352FCBDEC9DE432FACDE11E02227510FA8
:10030C00621F22CF4C3421F410E117BBC49A65C094
:10031C00453659F43CEAB9DE30E8B7DE34E0B5DEF8
:10032C0030E0B3DE10E3AADE58C04C3671F498DE30
:10033C003CEAABDE342F3670306EA7DE30E0A5DE43
:10034C0030E0A3DE10E39ADE48C0433789F4B2E014
:10035C0005D0B1E003D0B0E001D0F6CE30E395DEAD
:10036C0030E093DE3B2F91DE8FDE432F72DE08955B
:10037C004D3659F43CE489DE362F87DE352F85DE89
:10038C0030E083DE1FEF7ADE28C04A3359F468DE92
:10039C00C42F66DED42F64DEE42F442710D01FEF69
:1003AC006DDE1BC04E32B1F45BDEC42F59DED42F90
:1003BC0057DEE42F55DE03D01FEF60DE0EC03C2F5E
:1003CC0064DE3D2F62DE3E2F60DE342F5EDE4F2F6B
:1003DC0040DE08954FE33DDEB7CE4DE03ADEB4CEBD
:1003EC000000133029F0000000001A951330E9F7D3
:0203FC00089562
:00000001FF
